:020000040000FA
:02000000712D60
:08000800FF00030E8301FE005E
:100010008312031300308A0023308100A20A0530C6
:1000200022020318A2012114A30F1928A40F1928D2
:10003000A1145708003E03193828481C3628831697
:10004000031339308500831203138514C72201304E
:10005000D12200001E30A50085100730D122851462
:100060000630D122A50B2C2885105028C72239280C
:10007000BC222E30A6000830FD00220803195820AB
:100080000130220203197420023022020319902049
:10009000033022020319AC20043022020319C820C5
:1000A000373085000B117E0E8300FF0E7F0E090096
:1000B000E420A60B58286121E4206721E420752163
:1000C000E420C022E42085196D2810304502031871
:1000D0006B28C50A7328421573284508031972282E
:1000E000C503732842110800FD20A60B7428612166
:1000F000FD206721FD207521FD20C022FD208519EE
:1001000089281030460203188728C60A8F28C2158E
:100110008F28460803198E28C6038F28C2110800AD
:100120001621A60B90286121162167211621752121
:100130001621C02216218519A52810304702031860
:10014000A328C70AAB284216AB2847080319AA28D8
:10015000C703AB28421208004821A60BAC28612136
:1001600048216721482175214821C022482185194D
:10017000C128103043020318BF28C30AC7284214FD
:10018000C72843080319C628C303C728421008001C
:100190002F21A60BC82861212F2167212F2175212E
:1001A0002F21C0222F218519DD2810304402031889
:1001B000DB28C40AE328C214E32844080319E22810
:1001C000C403E328C210080001082B02031CFD141D
:1001D00001082F02031C7D1501083302031C7D1644
:1001E00001083702031CFD16831603137D088500E2
:1001F0008312031336308500080001082702031C10
:100200007D1401083002031C7D1501083402031C13
:100210007D1601083802031CFD16831603137D08A2
:100220008500831203133530850008000108280279
:10023000031C7D1401082C02031CFD140108350267
:10024000031C7D1601083902031CFD1683160313D7
:100250007D088500831203133330850008000108F0
:100260002902031C7D1401082D02031CFD14010842
:100270003102031C7D1501083A02031CFD1683168A
:1002800003137D08850083120313273085000800BF
:1002900001082A02031C7D1401082E02031CFD1410
:1002A00001083202031C7D1501083602031C7D166D
:1002B000831603137D08850083120313173085000E
:1002C000080003103B0DC9006E21CC00080003108C
:1002D0003B0D013EC9006E21CD00080001308A00AF
:1002E0004908793E03188A0A82004C088A004D08A2
:1002F00082000134B9340134C1340134C9340134C9
:10030000D1340134D9340134E1340134E9340134D5
:10031000F4340134F834023404340234083402343E
:1003200014340234183402342434023428340234AD
:10033000343402343834023444340234483402341D
:10034000543402345834023464340234683402348D
:1003500074340234783402348434023488340234FD
:100360009434023498340234A4340234A83402346D
:10037000B4343D18BE290630BB00B62A0130BB009C
:10038000B62A3D18C6290030BB00B62A0230BB0091
:10039000B62A3D18CE290030BB00B62A0330BB0078
:1003A000B62A3D18D6290430BB00B62A0330BB005C
:1003B000B62A3D18DE290030BB00B62A0530BB0046
:1003C000B62A3D18E6290730BB00B62A0030BB002C
:1003D000B62A3D18F22900304B070319F129CB0B3F
:1003E000B62AB62ABB01B62A3D08C100BB0AB62A06
:1003F00041083D06031DFE29BB01B62A3D184010E9
:100400003D1C4014BB0AB62A3D08C100BB0AB62AEF
:1004100041083D06031D0E2ABB01B62A3D183F12B6
:100420003D1C3F16BB0AB62A3D08C100BB0AB62ACE
:1004300041083D06031D1E2ABB01B62A3D18BF1107
:100440003D1CBF15BB0AB62A3D08C100BB0AB62A2F
:1004500041083D06031D2E2ABB01B62A3D183F1157
:100460003D1C3F15BB0AB62A3D08C100BB0AB62A8F
:1004700041083D06031D3E2ABB01B62A3D18BF10A8
:100480003D1CBF14BB0AB62A3D08C100BB0AB62AF0
:1004900041083D06031D4E2ABB01B62A3D183F10F8
:1004A0003D1C3F14BB0AB62A3D08C100BB0AB62A50
:1004B00041083D06031D5E2ABB01B62A3D18BE1247
:1004C0003D1CBE16BB0AB62A3D08C100BB0AB62AAF
:1004D00041083D06031D6E2ABB01B62A3D183E1297
:1004E0003D1C3E16BB0AB62A3D08C100BB0AB62A0F
:1004F00041083D06031D7E2ABB01B62A3D18BE11E8
:100500003D1CBE15BB0AB62A3D08C100BB0AB62A6F
:1005100041083D06031D8E2ABB01B62A3D183E1137
:100520003D1C3E15BB0AB62A3D08C100BB0AB62ACF
:1005300041083D06031D9E2ABB01B62A3D18BE1088
:100540003D1CBE14BB0AB62A3D08C100BB0AB62A30
:1005500041083D06031DAE2ABB01B62A3D183E10D8
:100560003D1C3E14BB0AB62ABB014A1408004210C7
:10057000C210851E421408003D1085193D14080064
:100580003C083B02031CC62A3B08BC00080048107C
:10059000D7030310D60CD50CD40CD30C0318481475
:1005A0000800CE00CE0BD22A0800D401D501D60116
:1005B000A030D300D109511C54145118D4144F1E2B
:1005C00054154F1AD415CF1D5416CF19D4164F1DDC
:1005D00054174F19D417CF1C5514CF18D5144F1CCE
:1005E00055154F18D515D01E5516D01AD516501EB4
:1005F0005517501AD517D01D5614D019D614501DA2
:1006000056155019D615D01C5616D018D616501C93
:1006100056175018D6172130D7000800D801D90135
:100620000830DA000310DC0CD90DD80DDB0CD90D25
:10063000D80DDA0B122B0800DD000000DD0B1D2B9E
:100640000800E50A65080F3C0319E5016508D200BA
:10065000FC010800E5036508013E031D322B0E3046
:10066000E500D200FC0108003E08E500D200F13EA2
:10067000031C3E2B0E30E5026508372BFC010800F9
:10068000DE002110211C422BDE0B412B0800650AE5
:10069000E700DC00DB010E235808E7005908E800FA
:1006A000E901E0306C18E900FF309524E701E8012A
:1006B000E9010130952408000530DF00F330E00047
:1006C0000310650DFC008B13E6258B17E200031465
:1006D000650DFC008B13E6258B17E0006208DF0038
:1006E000080021305F02031D792B60087C07A223DC
:1006F0008B2B8B130A08E3005F087B07F3000310C2
:1007000060087C07F4000318F30AED25E400630891
:100710008A0064088B17FC0F8E2BFB0A08008316D7
:1007200003139C18912B8B131C157C089B007A08D3
:100730009A0055309D00AA309D009C148B1783129F
:10074000031308008B13831603139C18A52B1C118D
:100750009B009C131C141A08831203138B170800A8
:100760009730A223EC000800B0236C1CB92B6C104E
:10077000BA2B6C149730FC006C08FA008F234723C7
:10078000472308005C23FC01FB017123E600E6130C
:100790007123EB00EB0A7123ED004A1CEB2B0730B1
:1007A0003F02031DD62B3423CA01C22BBF08031DF1
:1007B000EB2B20303E020319212321303E02031986
:1007C0002A2300303E020319E5010C303E020319D2
:1007D000B423CA01C22B42080319052C472347231F
:1007E000033042020319AF2D0C3042020319B42327
:1007F0004218FD2BC218012CC22B2123472347236B
:10080000F02B2A2347234723F02B063066020319D7
:100810002C241330660204308A0003193D2403306F
:100820008A001530660206308A000319112603304B
:100830008A005708003E031D292CA11C292CA11059
:100840006C1C242C2123C22B0730CF005208D0006F
:10085000D522ED0BCD2BC22B7123E7007123E800CD
:100860007123E9001F306905EE00EE0AEE0DEE0D72
:100870006B089524EE0B382C08007123E7007123D8
:10088000E8000F306805EF000F306F02031D4D2C9C
:10089000E701E801E90195248A2CE71B692C671F11
:1008A000682C3408BA002B08B4003908AB003508AE
:1008B000B9002F08B5003808AF003708B800330872
:1008C000B700B30140306718B307A030E718B3078B
:1008D000822C671F822C3708B3003808B7002F0816
:1008E000B8003508AF003908B5002B08B900340846
:1008F000AB003A08B400BA0140306718BA07A0301C
:10090000E718BA076B08402342188A2C4A188A2C29
:10091000EF0B4D2C0800700D700D701A013AF01A93
:10092000013AF019013AF0000800EA00B301E71BB0
:10093000B309B701E71AB709B801E719B809AF0158
:10094000E718AF09B501E81BB509B901E81AB909FB
:10095000AB01E819AB09B401E818B409BA01E91B05
:10096000BA09A901AA01AE01A801B101B201A7010A
:10097000AD01B601AC01B0016A08402308000230A5
:100980003B02031C0301E7000030E800013095241E
:1009900042080319F92CBC01BB015708003E031D96
:1009A000C82C4208E800E70101309524CF0103304C
:1009B00042020319AF2D4218E52CC218E92C421946
:1009C000ED2CC219F12C421AF52C2030D000D52282
:1009D000C82C2130D000D522C82C1030D000D52210
:1009E000C82C1130D000D522C82C0C30D000D52214
:1009F000C82C4A1CBF2CCA01F030E700E8017F3048
:100A00009524E701E8013F309524F030E700E80144
:100A10007F3095243E08E7003F08E800FF3095242A
:100A2000FF309524BC01BB01BF2C59250330420285
:100A30000319AF2D42185925013071020319362DC3
:100A40000230710203193B2D033071020319402D4E
:100A5000043071020319462D0530710203194C2D23
:100A6000063071020319512D5925162DE701C030AA
:100A7000E800E901562D0C30E700E800E901562DA9
:100A80000C30E700CC30E800E901562DCC30E7000F
:100A9000E9000C30E800562DCC30E700E800E80013
:100AA000562DCF30E700E9003C30E800FF309524B8
:100AB000162DE40A8B245530E700E800E900FF30EA
:100AC0009524AA30E700E800E900FF309524421899
:100AD000592D700823076407F100F10C0730F10568
:100AE000080085018101E501D701C001BF01BE01F8
:100AF000C101BB01BC01CA01A201A301A4010730CD
:100B00009900831603138230810070308F049F0197
:100B100083120313C2011D30F0008B168B17FF30B8
:100B2000E700E800E900FF309524FF309524FF300E
:100B30009524FF309524E701E801E901FF30952471
:100B4000FF309524FF309524B0234208E800FF30A1
:100B50009524FF309524F20142080319C22BE701C6
:100B6000720ADC00DB010E235808E8005908E9008E
:100B7000E80CE90CE80CE90CE80CE90CE80CE90CD1
:100B8000FF309524FF3095244218D825C218DE2561
:100B9000421ACB2DAF2D003072020319C22B013047
:100BA00072020319BF2C023072020319152DAF2DEA
:100BB000F20A7208033C0319F2010800F2037208FA
:100BC000013E031DE52D0230F20008005F088A0097
:100BD0007C08600703188A0A82000A08E300730889
:100BE0008A00740882000634653406348034063482
:100BF0008F3406349E340634A7340634C5340634A4
:100C0000CE340634EC340634FB3407344034073435
:100C100047342134013421343D34213449342134E2
:100C20008B3403308A007123E7007123E8007123BD
:100C3000E9003F306905EE00EE0DEE0D3330840023
:100C4000671B5D26671F612637308400671A5D26A3
:100C5000671E61263830840067195D26671D61268E
:100C60002F30840067185D26671C612635308400AC
:100C7000681B5D26681F612639308400681A5D266E
:100C8000681E61262B30840068195D26681D612668
:100C90003430840068185D26681C61263A30840070
:100CA000691B5D26691F61266B08402342185C2E74
:100CB0004A185C2EEE0B1E2E0800800A03198009CC
:100CC00008008008031D80030800133440340C34EE
:100CD000BF340134B0340934DF340134D034093442
:100CE000FF340134F03409343F34013430340934F2
:100CF0005F340134503409347F34013470340934A2
:100D000006343034043480340034803420340234E7
:100D100000340834083400340234203400341534EC
:100D200010340434553455345F34003400341F34E7
:100D30000034C0340F34FF34FF34DF34153403344F
:100D40000234553455347F34003400343F34153484
:100D500003340934043400341F34043400341F34A1
:100D60001C3410341F34783470345F34E134E1348F
:100D7000DF34833487349F3402340E341F3400341C
:100D800008341F34003400343F3406343034023425
:100D9000553455344034AA34AA34A034063430349F
:100DA00009348034003440344034003480342034FA
:100DB0000134003410340234003408340434003474
:100DC0000434083400340234103400340134203444
:100DD00000340034C0340034063410340434113488
:100DE0001134003422342234203444344434403426
:100DF000883488348034063417341634113411346E
:100E0000003422342234203444344434403488348E
:100E100088348034113411340034223422342034A4
:100E200044344434403488348834803411341134A8
:100E3000003422342234203444344434403488345E
:100E400088348034443444344034223422342034CE
:100E500011341134003488348834803444344434B8
:100E60004034223422342034113411340034883494
:100E7000883480344434443440342234223420349E
:100E8000133440340234FC340934F3340934133459
:100E900080340C34D53409345A340934DF340934FD
:100EA0005A340934D534093450340934753409348A
:100EB000FA3409347F340934FA3409347534093486
:040EC000F0340934CD
:02400E00C430BC
:10420000FF000600050013000034003420340034A1
:104210000034803400340234003400340834003474
:10422000003420340034003480340034023400344C
:104230000034083400340034203400340034803436
:10424000003400344034003400341034003400347E
:104250000434003400340134003400340034403479
:10426000003400341034003400340434003400349A
:1042700001340034003400344034060010000300E0
:1042800092344934203449342434803424349234F0
:10429000403406000500150000340034203400349A
:1042A00000348034003402340034003408340034E4
:1042B00000342034003400348034003402340034BC
:1042C00000340834003400342034003400348034A6
:1042D00000340034003400340034003400344034FE
:1042E0000034013400340034043400340034103419
:1042F00000340034403400340134003400340434D9
:1043000000340034103400340034403400340034BD
:1043100000340034003406001000030092344934A5
:1043200020342434923440344934243480340034EA
:00000001FF
